:020000040800F2
:10000000C006002051020008E70E0008790E000823
:10001000E50E00086B040008AD10000800000000A9
:10002000000000000000000000000000EB0E0008CF
:100030006D04000800000000E90E0008ED0E000845
:100040006B0200086B0200086B0200086B020008DC
:100050006B0200086B0200086B0200086B020008CC
:100060006B0200086B0200086B0200086B020008BC
:100070006B0200086B0200086B0200086B020008AC
:100080006B0200086B0200086B0200086B0200089C
:100090006B0200086B0200086B0200086B0200088C
:1000A0006B0200086B0200086B0200086B0200087C
:1000B0006B0200086B0200086B0200086B0200086C
:1000C0006B0200086B0200086B0200086B0200085C
:1000D0006B0200086B0200086B0200086B0200084C
:1000E0006B0200086B0200086B0200086B0200083C
:1000F0006B0200086B0200086B0200086B0200082C
:100100006B0200086B0200086B0200086B0200081B
:100110006B0200086B0200086B0200086B0200080B
:100120006B0200086B0200086B0200086B020008FB
:100130006B0200086B0200086B0200086B020008EB
:100140006B0200086B0200086B0200086B020008DB
:100150006B0200086B0200086B0200086B020008CB
:100160006B0200086B0200086B0200086B020008BB
:100170006B0200086B0200086B0200080000000020
:100180006B0200086B0200086B0200086B0200089B
:100190006B0200086B0200086B0200086B0200088B
:1001A0006B0200086B0200086B02000800F002F806
:1001B00000F03EF80AA090E8000C82448344AAF1C3
:1001C0000107DA4501D100F033F8AFF2090EBAE8C1
:1001D0000F0013F0010F18BFFB1A43F0010318477B
:1001E000780F0000980F0000103A24BF78C878C13B
:1001F000FAD8520724BF30C830C144BF04680C602D
:10020000704700000023002400250026103A28BF74
:1002100078C1FBD8520728BF30C148BF0B60704778
:100220001FB500F07CFF00F0D5F81FBD10B510BD64
:1002300000F0EDF81146FFF7F3FF00F063FF00F068
:100240000BF903B4FFF7F2FF03BC00F0D9F800008C
:100250000948804709480047FEE7FEE7FEE7FEE75A
:10026000FEE7FEE7FEE7FEE7FEE7FEE70448054996
:10027000054A064B70470000910F0008AD010008C9
:10028000C0000020C0060020C0020020C0020020E4
:1002900053EA020C00F069802DE9F04B4FF00006A4
:1002A000002B1FBFB3FA83F503FA05F424FA05F611
:1002B0005E4012BF1643B2FA82F502FA05F4C5F1A8
:1002C00020051EBF22FA05FC44EA0C04203556EA3C
:1002D000044C4FEA144418BF641C4FF000084FF060
:1002E0000009904271EB030C39D3002919BFB1FA10
:1002F00081F701FA07F6B0FA80F700FA07F6C7F1BE
:1003000020071EBF20FA07FC46EA0C062037B6FB82
:10031000F4FCA7EB0507103F07F01F0BCBF12006FD
:100320000CFA0BFB2CFA06F644BFB3460026202F2E
:10033000A4BF5E464FF0000B5BEA060C08BF4FF00F
:10034000010B19EB0B09ABFB027C48EB0608C01B49
:1003500006FB02CC0BFB03CC71EB0C01C1E70B4697
:10036000024641464846BDE8F08B13B54FF0000009
:100370004FF00001AFF30080BDE81C4070474FF024
:10038000000200B5134694469646203922BFA0E8E5
:100390000C50A0E80C50B1F12001BFF4F7AF0907F1
:1003A00028BFA0E80C5048BF0CC05DF804EB8900E2
:1003B00028BF40F8042B08BF704748BF20F8022B25
:1003C00011F0804F18BF00F8012B7047704770473D
:1003D0007047000070B5064C7C44064D7D4403E038
:1003E000206820448047241DAC42F9D170BD000034
:1003F0009C0D00009C0D000000487047600000202C
:1004000001491820ABBEFEE7260002007047754682
:10041000FFF7F2FFAE4605006946534620F007009D
:10042000854618B020B5FFF721FFBDE820404FF00A
:1004300000064FF000074FF000084FF0000B21F0CE
:100440000701AC46ACE8C009ACE8C009ACE8C0099B
:10045000ACE8C0098D46704710B50446AFF3008084
:100460002046BDE81040FFF7ECBEFEE7704772B6CD
:10047000FEE700002DE9F84FDFF8F8A10022012483
:1004800003254FF00F090AF1040BAAF1040E00BF77
:100490000B6804FA02F63340B34270D10F7907F0CB
:1004A0000307012F01D0022F16D187684FEA4208B7
:1004B00005FA08FC27EA0C07D1F80CC00CFA08FC76
:1004C0004CEA070CC0F808C04768B7430E79C6F37A
:1004D000001696403E4346600E79F643B6070AD0B2
:1004E000C7684FEA420C05FA0CF6B7438E6806FA65
:1004F0000CF63E43C6600E7906F00306022E10D1BC
:10050000D60800EB8608D8F8206057074FEAD76C6A
:1005100009FA0CF7BE430F6907FA0CF73743C8F81E
:10052000207006684FEA420C05FA0CF7BE430F79BB
:1005300007F0030707FA0CF7374307604E6816F415
:10054000403F1CD04C4E376847F4804737603668D0
:1005500022F0030706F480460096484E07EB060C8F
:10056000DCF8086897073F0F09FA07F826EA08063B
:10057000DFF80C81404503D14FF0000841E072E004
:10058000DFF80081404502D14FF0010839E0DFF883
:10059000F880404502D14FF0020832E0DFF8EC80ED
:1005A000404502D14FF003082BE0DFF8E4804045DE
:1005B00002D14FF0040824E0DFF8D880404502D192
:1005C0004FF005081DE0DFF8D080404502D14FF024
:1005D000060816E0DFF8C480404502D14FF0070856
:1005E0000FE0DFF8BC80404502D14FF0080808E07A
:1005F000DFF8B080404502D14FF0090801E04FF02C
:100600000A0808FA07F848EA0608CCF80888DAF871
:1006100000605746D1F804C09E435FEACC2C00D559
:100620001E433E60DBF800605F46D1F804C09E4385
:100630005FEA8C2C00D51E433E60DEF800607746F2
:10064000D1F804C09E435FEA8C3C00D51E433E6057
:10065000084F083F3E68D1F804C09E435FEACC3C97
:1006600000D51E433E60521C102AFFF411AFBDE8B6
:10067000F88F0000083C014044380240003001403F
:10068000000002400004024000080240000C02404A
:10069000001002400014024000180240001C0240FA
:1006A000002002400024024001488068704700009A
:1006B0000000002002488168027811448160704780
:1006C000000000200B4810B5016841F40071016082
:1006D000016841F480610160016841F4807101604A
:1006E000032000F061F8002000F006F800F024F884
:1006F000002010BD003C024070B50D4D04464FF483
:100700007A712878B1FBF0F00A490968B1FBF0F082
:1007100000F036FB48B9102C07D200222146501EAB
:1007200000F022F800206C6070BD012070BD000058
:10073000000000200C0000200A4808B5016841F4C0
:1007400080410160006800F4804000900548001F6F
:10075000016841F080510160006800F08050009015
:1007600008BD000044380240F0B40E4B1B680C4634
:10077000C3F30223C3F10705042D00D90425191D75
:10078000072901D2002300E0DB1E012606FA05F14D
:10079000491E214099409E40761E16403143F0BCD0
:1007A00000F098BC0CED00E0064900F00702086874
:1007B0004FF6FF03184040EA0220034A1043086046
:1007C000704700000CED00E00000FA052DE9F84349
:1007D0001748016841F0805101600068154F00F032
:1007E0008050012600903E64FFF75EFF05464FF4FF
:1007F0007A78114C05E000BFFFF756FF401B4045DB
:100800000DD86068C003F7D57E64FFF74DFF05463D
:10081000464607E0FFF748FF401BB04202D90320DD
:10082000BDE8F88360688003F4D50020F8E7000095
:100830004038024000000E42007000402DE9F047B1
:100840000E46050065D0DFF81481D8F80000F7B235
:1008500000F00F00B04207D288F80070D8F800000E
:1008600000F00F00B04254D128683D4C810712D5EA
:10087000400703D5206840F4E05020602878000746
:1008800003D5206840F4604020602068A96820F00B
:10089000F000084320602878C0072DD030496868F0
:1008A0000839012812D0022813D0032811D0096872
:1008B000890700292DDA216821F003010143216015
:1008C000FFF7F2FE814641F2883A0EE0096889039B
:1008D000EFE709688901ECE7FFF7E6FEA0EB090105
:1008E000514502D90320BDE8F0872068696800F00F
:1008F0000C00B0EB810FEFD1D8F80010404601F0AA
:100900000F01B14207D90770006800F00F00B04234
:1009100001D00120E7E72878400705D52068E9687D
:1009200020F4E050084320602878000706D52068AE
:10093000296920F4604040EAC100206000F038F8E6
:100940002168084AC1F30311515CC8400649086098
:1009500006480068FFF7D0FE0020C4E7003C0240D4
:1009600008380240281100080C0000200400002074
:100970000448054900680968044AC1F38221515CB2
:10098000C84070470C0000200838024038110008A9
:100990000448054900680968044AC1F34231515CC2
:1009A000C84070470C000020083802403811000889
:1009B000154810B5006810F00C02144813D0144903
:1009C000042A0FD0082A0ED10F4C241F2268236856
:1009D00002F03F025B0207D52068C0F38810A0FB3D
:1009E000010106E0084610BD2168C1F38811A1FB92
:1009F00000010023FFF74CFC2168C1F30141491CB1
:100A00004900B0FBF1F010BD083802400024F400AA
:100A100040787D012DE9F84F04006ED02078DFF892
:100A20004C93C007A9F104054AD009F104000168FC
:100A3000C1F38101012908D00068C0F381000228B8
:100A40000AD1D9F80000400206D52868800337D5BE
:100A500060680028E1D033E06068B0F5803F10D0D6
:100A6000B0F5A02F286810D020F4803028602868C6
:100A700020F4802028606068A8B1FFF715FE0646C4
:100A80000DE0286840F48030F4E740F480202860CE
:100A9000F7E700BFFFF708FE801B642873D82868BB
:100AA0008003F7D50CE0FFF7FFFD064605E000BF29
:100AB000FFF7FAFD801B6428F0D828688003F7D47C
:100AC0002078DFF8AC8280074FF0000A3ED5A748B7
:100AD000001D016811F00C0F08D00068C0F3810000
:100AE00002280BD1D9F80000400207D428688007FB
:100AF00016D5E068012800D112E033E1E068B8B112
:100B00000120C8F80000FFF7CFFD064605E000BF52
:100B1000FFF7CAFD801B0228C0D828688007F7D5D8
:100B20002868216920F0F80040EAC10028600DE043
:100B3000C8F800A0FFF7B8FD064604E0FFF7B4FDD3
:100B4000801B02281FD828688007F7D42078000768
:100B500022D5864F87486169703771B101210160E4
:100B6000FFF7A2FD064604E0FFF79EFD801B02286A
:100B700009D838688007F7D50EE0C0F800A0FFF765
:100B800093FD064605E082E0FFF78EFD801B0228FC
:100B90007DD838688007F7D42078400768D5DFF81B
:100BA000CCB100270BF13C0BDBF80000C0000BD4EC
:100BB000DBF8001041F08051CBF80010DBF80000AA
:100BC000012700F0805000906B4E3068C00510D4B3
:100BD000306840F480703060FFF766FD009005E0FB
:100BE000FFF762FD0099401A022850D83068C0050E
:100BF000F6D55E4EA0686C3601280FD00528306807
:100C000010D020F001003060306820F00400306027
:100C1000A068B8B1FFF748FD00900FE0306840F0E1
:100C20000100F4E740F004003060F7E7FFF73CFD17
:100C30000099411A41F28830814266D830688007B5
:100C4000F4D50EE0FFF730FD009007E0FFF72CFD34
:100C50000099411A41F28830814256D830688007A5
:100C6000F4D42FB1DBF8001021F08051CBF8001044
:100C7000A069C8B33D49091D0968C1F38101022972
:100C80004AD00228504607D0C8F8600000E03CE097
:100C9000FFF70AFD04463BE04746C8F86000FFF74F
:100CA00003FD064605E000BFFFF7FEFC801B02289F
:100CB0002BD828688001F7D4D4E907010843A16A3A
:100CC0002E4A490802EB0141626A41EA8211084357
:100CD00094F82C1040EA0161C9F800100120386630
:100CE000FFF7E2FC044606E03EE000BFFFF7DCFC55
:100CF000001B022809D828688001F7D534E000BF1E
:100D0000FFF7D2FC001B022802D90320BDE8F88FB0
:100D100028688001F4D427E00128F7D0D9F8000032
:100D2000E26900F4800191421CD1226A00F03F0187
:100D3000914217D147F6C071626A0140B1EB821F40
:100D400010D1A26A4FF0FF3300F4403103EB52029E
:100D5000B1EB024F06D194F82C1000F07060B0EBAC
:100D6000016F01D00120D1E70020CFE70438024015
:100D700000004742800E4742007000400000FFFF25
:100D800010B5401EB0F1807F01D3012010BD4FF09F
:100D9000E02460610F21601700F09CF90020A06141
:100DA00007202061002010BD70B5040004D094F825
:100DB0003D00002510B106E0012070BD84F83C50D4
:100DC000204600F023F8242084F83D002068C16804
:100DD00021F40051C160204600F0E2F8206801696A
:100DE00021F4904101612068416921F02A014161AB
:100DF0002068C16841F40051C1602564202084F856
:100E00003D0084F83E00002070BD000010B586B0A3
:100E1000044614216846FFF7B2FA14492068884254
:100E200021D113480021026842F0100202600068DC
:100E300000F0100005900E481438026842F00102DC
:100E40000260006800F0010005904FF4C06000905F
:100E50000220CDE901010320039007200490694698
:100E60000448FFF707FB06B010BD0000001001406A
:100E70004438024000000240FEE70000094808B57F
:100E8000016841F080010160016801F0800100917A
:100E9000016841F001010160006800F0010000906C
:100EA00008BD0000303802400C4810B50A49016006
:100EB0004FF4E1314160002181600C22C160C0E942
:100EC00004128161C161FFF76FFF002803D0BDE804
:100ED0001040FFF7CCBA10BD0010014010000020F8
:100EE0007047FEE7FEE7FEE770477047FFF7E2BB9B
:100EF00030B593B030216846FFF741FA14210CA8B1
:100F0000FFF73DFA20480025016841F0805101605B
:100F1000006800F0805011901C48016841F4404185
:100F200001600068022400F4404011900120039009
:100F300010200490009406940820CDE90750B420B6
:100F4000CDE9090404200B906846FFF763FD08B162
:100F500072B6FEE7FFF73AFC08B172B6FEE70CA9DD
:100F60000F2081E831004FF4A0500F904FF48050D3
:100F7000109005210CA8FFF761FC002801D072B683
:100F8000FEE713B030BD0000403802400070004062
:100F90000248016841F470010160704788ED00E08B
:100FA00070B5044600680169E26821F440511143BC
:100FB00001612169A068E26908436169114308433E
:100FC0002168CA6849F20C639A430243CA602068E8
:100FD0004169A26921F4407111434161314920689E
:100FE000884202D03049884202D1FFF7D1FC01E0AB
:100FF000FFF7BEFCE2690023192164253226B2F511
:10100000004F626828D0A0FB0101930F9200FFF708
:101010003FF90146B0FBF5F06FF01802504301EBC9
:10102000800006EB0010B0FBF5F000F0F002B1FB21
:10103000F5F002EB0012B1FBF5F06FF01803584326
:1010400001EB800006EB0010B0FBF5F000F00F00A4
:1010500021681044886070BDA0FB010192185B41BB
:10106000FFF716F90146B0FBF5F00201B1FBF5F010
:101070006FF01803584301EB800006EBC000B0FB93
:10108000F5F000F0F80002EB4002B1FBF5F0584338
:1010900001EB800006EBC000B0FBF5F000F00700AC
:1010A000D6E700000010014000140140FEE70000F8
:1010B000024901608021416070470000481100082A
:1010C00000B50A46FFF7F4FF01498260016000BDE8
:1010D000541100080907090E002804DB00F1E02084
:1010E00080F80014704700F00F0000F1E02080F855
:1010F000141D704701490248FFF7E2BF10000020AD
:1011000054000020FFF7DEFAFFF7F2FEFFF7B6FE0D
:10111000FFF7CAFEFFF7E4FEFFF7E3FEFCE74FF040
:101120004070E1EE100A704700000000000000006F
:10113000010203040607080900000000010203047D
:10114000000000000000000000000000000000009F
:1011500000000000000000007C11000800000020DA
:1011600010000000E80100088C11000810000020A9
:10117000B0060000040200087DFFFFFF0100000030
:0C11800010000000000000000024F4003B
:04000005080001AD41
:00000001FF
